S0080000666C617368E9
S11300000DC00BC00AC009C008C007C006C005C0A7
S113001004C003C002C001C000C01895F8940FE1E9
S113002001BD07E101BD00E0A89501BD00E005BFE9
S113003011241ABA1BBA17BA18BA14BA15BA11BAD3
S113004012BA13BE1FBC1EBC1BBE19BE1ABE18BEFC
S11300501AB81CBA1DB818B80FE50DBF02E00EBFE0
S1130060A1E6B0E081E090E001C01D920197E9F7BC
S1130070A0E6B0E0E4EDF0E081E090E003C0C895D4
S10D008031960D920197D9F700C0E4
S11300B444275527009749F02AE030E04F5F5F4F0B
S11300C421503040D9F70197B9F7952F842F08951B
S113008ACFE5D2E0CDBFDEBF8FEF84BBC8EED3E0AD
S113009A1FEF15BA8C2F9D2F08D015BB8C2F9D2FBF
S10D00AA04D0C851DC4FF5CFFFCF9E
S10400D40027
S9030000fc
